:020000040000FA
:06000000D7EF04F0000040
:020006000000F8
:08000800F2B20BD8F0B2FF00C8
:04001000F292110057
:08001800F0A01000F090028E30
:020020001000CE
:0E0022003BD88A981AB0FF001AB212001AAE2C
:1000300012001A500C0B05E0FE0E79D81AB0FF0022
:100040001200000E1B5C16E0FF0E1B5C13E0FE0EA0
:100050001B5C10E0FA0E1B5C0DE0AA0E1B5C04E1B9
:100060001D8C1D881E9E06D0FC0E1B5C05E11D9C90
:100070001D981E8E8A881200F50E0C5CD8B00D8E6D
:100080001B50DE6E0C2A3E0ED95C010EDA58D8B039
:1000900020EE40F00DAEEED712001A6A080E186E70
:1000A000010E196E010ED56EF2949E0ED76E176E6C
:1000B000580ED66E166ED58E20D8FEE61ED8FEE7F8
:1000C0001CD8FEE602E3192AD8801B32182EF6D778
:1000D00014D8FEE712D8FEE61834191A193001E3D5
:1000E0001A840BD8FEE709D8FEE601E21A8605D885
:1000F000FEE71A8ED59EF2941200F2B413D081500E
:100100000D0B1C6E81500D0B1C62F7D71CA407D081
:10011000D8981CB6D888D8901CB0D88012001A8005
:10012000060012001A82D59EF294060012001B6E81
:100130001A6A080ED56EF294FE0ED76E0C0ED66EAD
:10014000080E186E010E196E8A98D58EF2A4FED78D
:100150008A9AD59EF294010ED56E9E0ED76E580ED9
:10016000D66ED58E8A88C9DFFEE61B3203E3192AD4
:100170008A8A01D08A9AC1DFFEE7BFDFFEE6182E29
:10018000F4D7193202E38A8A01D08A9AB6DFFEE7F1
:10019000B4DFFEE68A8AB1DFFEE7AFDFFEE601E309
:1001A0001A88ABDFFEE71A8CD59EF29412004DEC54
:1001B00000F01AB0FF001AB205D01A500C0B02E181
:1001C000D8901200D8801200ED0E02D813E226500B
:1001D000AEDF1AB0FF001AB20DD01AAC0BD01AACB9
:1001E00009D01AB807D0E3DF05E2FA0E1B6202D08D
:1001F000D8901200D8801200D09CD082F26AF16AA6
:10020000F06A9E6AA16A9D6AA06AC26A926893684F
:100210009468956896680F0EC16E89688A688B68C5
:100220008C688D6AC30E926ECF0E936E946A8B9C0F
:10023000966AF86A92D881A4FED7D08EF19EF08E8D
:10024000F09CF288F086F0888B8C0C0E166EFE0EF9
:10025000176EA4D88B9E9C0E166EFF0E176E9ED83E
:100260008B8EB00E166E3C0E176E96D8F292070E5D
:10027000D56EF2948D0ED76E900ED66ED58EF2B4EA
:100280001CD0F0B2FF00F2A2FAD7D59EF2944DEC4A
:1002900000F01AB0FF001AB210D01AAE0ED01A50E9
:1002A0000C0B0BE1AA0E1B6203D01D8C1D8804D021
:1002B000FC0E1B6201D01E8E1D8ED59EF294F29212
:1002C0001DAE79D8F2921DAE3CD01DAC3AD0F29260
:1002D000F20EE8EC00F011E2D7EC00F00EE21B5059
:1002E000006ED7EC00F009E21B50016EAB0E00620D
:1002F00004D0830E016201D01D8AF292ED0EE8EC6B
:1003000000F005E2000EE8EC00F001E21D80F29240
:10031000F00EE8EC00F005E2020EE8EC00F001E27D
:100320001D82F292F30EE8EC00F005E20B0EE8EC11
:1003300000F001E21D86F292F40EE8EC00F001E21A
:100340001D848A98030E8D6E1D5048EC04F0F292C5
:10035000F090F092F28EF28C120000EE00F0030E9C
:10036000EE6AEA62FDD7040E036E8D6A956A8C6AA6
:10037000000000008B9200008B8200008D2A032E6B
:10038000F7D720EE40F010EE40F03E0E0E6E106EED
:10039000010E0F6E116E1200010E01D0080ED56E07
:1003A000F2941750D76E1650D66ED58EF2A4FED7A3
:1003B000D59EF2941200EE0E97EC00F01AB0FF00FA
:1003C0001AB212001AAC12004DEC00F01AB0FF0085
:1003D0001AB212001D8E1AAE12001A500C0B04E154
:1003E000EE0E1B6212001D8C1200000E0C5C03E16D
:1003F0000D9E8A88120012BE1200E6500B6EF29E0D
:10040000F29C0C060D9E8A88F28EF28C0DA817D0F5
:100410000900F5500B5CD8A40D860A2E04D00DA659
:100420000AD0800E0D163E0EE15C010EE258D8B0E7
:1004300010EE40F01200090E1F6E15DA08D1F00E12
:100440000B5C02E10D8CEFD7E00E0B5C04E1800E3B
:100450000D160D8AE8D7E10E0B5C0AE1800E0D1631
:100460000D886F0EF66E0A0EF76E070E0A6EDBD75A
:100470000DAA17D0760EF66E0A0EF76E0A680A2AD3
:100480000900FF0EF55CCDE0F5500B5CF8E18D0E38
:100490000A24F66E0A0EF76EE86AF7220900F55094
:1004A00020D0A30EF66E0A0EF76E0A680A2A09001B
:1004B000FF0EF55C0DE0F5500B5CF8E1AB0E0A2485
:1004C000F66E0A0EF76EE86AF7220900F55009D0B9
:1004D000700E0B5C0B5005E37F0E0B5CA2E2100E5E
:1004E0000B5C0A6EB20E0A24F66E0A0EF76EE86A0C
:1004F000F7220900F5501F6E94E67B0E1F5C91E217
:10050000129C129A12982B9C610E1F5C08E3146ACD
:100510001F50156E200E1F5C2C6E2B8C0ED1420EC0
:100520001F5C1CE30B6E570E1F5C01E37AD7D8905B
:100530000B3612882BBE0ED020BE0B2AD80E0B24F1
:10054000F66E090EF76EE86AF7220800F550156E90
:10055000146AF4D0000E156E146AF0D0180E1F5CE9
:1005600018E30B6E200E1F5C14E2220E0B24F66EB5
:100570000B0EF76EE86AF7220800F5500B6E0DBC03
:1005800006D02A1401E04DD70B502A1202E10B1CB1
:100590002A1669D9155201E144D7C00E145C04E152
:1005A0000DAC3FD70D9C50D1800E145C50E1225011
:1005B000236EC00E2014246E15500B6E0B1C2216D9
:1005C0000B500DAC2212229E229C240E2214D8A481
:1005D000228E120E2214D8A4228C209E209C090E5A
:1005E0002214D8A4208EC00E2214D8A4208C22500D
:1005F000236205D0C00E2014245C01E112D72250E2
:10060000156E20500B6E0B420B420B420B420B42FD
:100610000B40030B1412E00E135CD8B0128E0E5078
:10062000E96E0F50EA6E1450EE6E1550EE6E132AFE
:10063000E9500E6EEA500F6E000E0E5C030E0F585E
:10064000D8A0EFD63E0E0E6E010E0F6EEAD6900EBB
:10065000145C1FE12150276E2550286E090E1F5C87
:1006600002E1217813D00DBC07D0251401E0D9D6C2
:100670001550211A251202E1151C25162150275C60
:1006800001E1CFD695EC04F01DA0CBD62150156E1C
:10069000C2D7200E1F5C12E32B0E1F5C0FE221ACB1
:1006A00007D020AE0BD020BC09D01288128A128C41
:1006B0000B0E1F26D8D8155201E1B3D62B0E1F5CA6
:1006C00008E112B803D0C00E201403E10DBC01D024
:1006D00021741E0E1F5C03E01F0E1F5C03E1030E5E
:1006E0002A1421120A0E1F5C0CE3100E1F5C09E293
:1006F00020AE03D020BC01D01F2AB5D815523DE151
:1007000090D6360E1F5C39E320AE0BD00C0E20AC19
:1007100012D0300E22AE0FD0480E22AC0CD0540EA8
:100720000AD0000E20AC07D0180E22AE04D0240E42
:1007300022AC01D03C0E15267FD02C500B6E400E03
:100740000B5C1BE3600E0B5C18E222AE07D01F0EA1
:100750000B14600F156EA00E146E0FD022AC05D0D6
:100760001F0E0B14156E146A08D02BAC06D0205047
:100770002118800B02E02C50156E14BE21D0300ED3
:10078000155C0B6E11E33A0E155C0EE222AE04D03E
:10079000300E22BC500E03D022AC4ED0400E0B24A3
:1007A000156EA00E146E48D01B0E155C09E0090EE4
:1007B000155C06E02B0E155C03E02D0E155C3CE18C
:1007C000700E1214700838E0620EF66E0A0EF76EA4
:1007D0000A680A2A0900FF0EF55C2EE01550F55C48
:1007E000F8E1C00E221409E0C00802E1030E08D0AF
:1007F000010E22BE05D0020E03D020AE1DD0000E89
:10080000D8900A360A360A26020E0A24F66E0A0E16
:10081000F76EE86AF7220900F5500EE0156E320E09
:100820000A24F66E0A0EF76EE86AF7220900F55000
:10083000146EC00E145C08E00DBC148C14A8EBD62A
:1008400021500F0B1412E7D62C6A80A204D02C3E44
:10085000FCD711EF02F0020E8D6E155019D8829858
:1008600000008288DED52A0E1F24F66E0B0EF76E6E
:10087000E86AF7220800F550156E6C0E1F24F66E1C
:100880000B0EF76EE86AF7220800F550146E12009E
:100890008C6E956A000000008B9200008B82000035
:1008A000120095688D6A040E036E00EE04F08B90C2
:1008B0000000000083508362FDD78B80EE6E8D2A8E
:1008C000032EF5D78D6A029EE10E045C05E129D85E
:1008D000076A1DB007681BD0C10E045C02E18A885C
:1008E0001BD0C20E045C12E1F29EF29C8B9C070EA0
:1008F000D56EF2948D0ED76E900ED66ED58EF2A474
:10090000FED78B96000000008B86FF0005D0030EFB
:100910008D6E0750BDDF00D08B96000000008B86E7
:1009200012002150276E0550216E2150266E26425E
:100930002642264226422640070B266E8A50296E02
:100940008A98F29EF29CE4EC00F029A88A98F29230
:10095000F28EF28C06E32750216E2850256E1D90F2
:1009600012001D80120080B012001050E96E11506C
:10097000EA6EEE50146EEE50156E8D6A145088DFDC
:10098000010E8D6E155084DF829A0000828A130654
:10099000E950106EEA50116E000E105C030E1158F3
:1009A000D8A012003E0E106E010E116E1200000152
:1009B000FCEC00F0899A8AA804D0F5EC01F01366EB
:0809C000D2DF02BE6EDFF7D7A3
:0809C800000000000000000027
:1009D0000000000000000000607E3121324034241D
:1009E00033233525365E3726382A2C3C30293928E2
:1009F0002E3E2F3F3B3A2D5F27225B7B3D2B5D7DBB
:100A00005C7C0102030405060708090A0B0C0D0EA5
:100A10000F10111213141516178018191A811B1CA8
:100A20001D82001E1F88002021220023242500266D
:100A30002728A0A0A0A0A0A0A0A0A0A0A0A0A0A0A7
:100A4000A0A0A0A0A0A0A0A0A0C0A0A0A0C0A0A066
:100A5000A0C0A0A0A0C0A0A0A0A0A0A0A0A0A0A056
:100A6000A0A0838586888A8C8E901B092B2DFF146D
:100A700077E1F014F0777C111470716C697A7D75F0
:100A80006B72745A4A1F272F373F5E7EFF00100F8C
:100A9000130817181920283038395A5F1F272F37A5
:100AA0003F5E48838466696B6C61FF0240474F502C
:100AB00051531E3E3C3A38363741353F3D3B390EA7
:100AC00042040502002B017143322C2E7A736177A8
:100AD000441C346378646545461B3314766674722F
:100AE000471D2F6E62686779481A2D316D6A754906
:100AF0004A19174B6B696F4C4D15164E4F6C507061
:100B000051212427520C5354FFFF06030A55FF5668
:100B10001810202A222526281F07401123121329E6
:100B200008FF204080081004010201020408102080
:100B3000804020100D8D3C3E09892F2B2D2A2090BE
:100B40008384858687808182831B303132333435BC
:100B5000363738392E868C8B8A8F00878584888E2D
:100B6000A0A1A2A3A4A5A6A7A8A9AAAB80808080C3
:100B700080809090909000A0000000A000000000F5
:100B800000A0C0C0C0C0C0A0A0A0B0100000000065
:100B900000000000000000B0A0A0A0A0A0A0A0A0A5
:0E0BA000A0A0A0A0A0A0A0A0A0A0A0A0A0A087
:020000040030CA
:0100010004FA
:010002001AE3
:010003001EDE
:010005008179
:010006008178
:00000001FF
